:03F0000002F00813
:03F0610002F003B7
:05F0030012F08B80FEFD
:04F06400AA82AB834E
:05F068001ABAFF011BB4
:0EF06D00C3E49A74808BF063F08095F0500F2E
:04F07B007CB07D04E4
:05F07F001CBCFF011D97
:06F08400EC4D70F780DE88
:01F08A002263
:0AF08B0090FE00E0FAC2A875E1044F
:0BF0950090DF3BE0FBBB01F875E103DE
:0AF0A00090DF3BE0FBBB13F87B00A0
:09F0AA008A047D000CBC00010D7C
:0EF0B3008B067F00C3EE9CEF64808DF063F04F
:05F0C1008095F0501ADB
:03F0C6003089FD91
:0EF0C90090DF3BE0FCBC13F8C2898B040B8C7B
:09F0D700827583FEE0F5D980CAC0
:0AF0E00090DF3BE0FABA130280F65D
:02F0EA00A5225D
:06F03700E478FFF6D8FDAD
:08F015007900E94400601B7A58
:05F01D000090F0F07806
:03F02200007593E3
:0AF0250000E493F2A308B80002050E
:08F02F0093D9F4DAF27593FFA6
:08F03D007800E84400600A7944
:03F04500007593C0
:06F0480000E4F309D8FC0E
:08F04E007800E84400600C7931
:0BF0560000900000E4F0A3D8FCD9FA01
:03F0080075810708
:0AF00B0012F0ECE582600302F0034E
:04F0EC007582002207
:00000001FF
